:100000000C942A001895000018950000189500001F
:100010000C940F0D1895000018950000189500001D
:10002000189500000C94A70C189500001895000076
:10003000189500001895000018950000189500000C
:1000400018950000189500001895000018950000FC
:10005000189500008FE181BD87E181BD8FE58DBFDF
:10006000C0E4E8E34E2E84E08EBFD4E0F4E05F2EDF
:10007000EEEFF3E0A0E6B0E088278D933197E9F743
:1000800089E189B988E18AB90E94BE0E66248A9AFC
:100090008B9AA09AA19A889AD39AD49AD59AEAEB85
:1000A000F0E080E40E94100F58E0C895802D0E9477
:1000B0000A0F31965A95C9F704C0040E0A0A0A0AB3
:1000C0000E20EEEDF0E088E40E94100F58E0C89595
:1000D000802D0E940A0F31965A95C9F704C0040E6C
:1000E0000E0E0E0E0E20E2E0F1E080E50E94100FF1
:1000F00058E0C895802D0E940A0F31965A95C9F78D
:1001000004C004040404150E0420E6E2F1E088E5CE
:100110000E94100F58E0C895802D0E940A0F31965A
:100120005A95C9F704C020111F1F1F1F1F2083E00D
:1001300086B9379A85E083BF8C9A8D9A81EA8FBD04
:1001400082E08EBD85E085BD88E082BD789489B768
:10015000816089BF89B7806489BF882783BF88276A
:1001600085BD929A939AA898A998DB98DC98DD9817
:10017000909880E090E09BBD8ABD80E08093B000C5
:1001800080E08093610080E090E0A4EAB0E08D938D
:100190009C9380E08093AA0080E090E0ABEAB0E01E
:1001A0008D939C9380E08093E80080E08093E90049
:1001B00080E08093EA0080E090E0A1EFB0E08D93D2
:1001C0009C9380E08093C7000E94A30E8FE711E00C
:1001D0000E94B20EECE2F7E20E949A0E8FEB11E061
:1001E0000E94B20EE6E4F7E20E949A0E8CE00E94B2
:1001F000100F0E943A0FA1E6B0E00C93009161004D
:10020000003011F00C9406010C9408010C94F900D4
:100210000E94A30E84E690E00E94610F709160003E
:100220007F77709360008FEB17E00E94B20EEEE5CF
:10023000F7E20E949A0E709160007F7B70936000DD
:100240008FE711E00E94B20EE6E6F7E20E949A0EF6
:100250008CE00E94100F0E943A0FA1E6B0E00C93D0
:1002600000916100043011F00C944801709160001D
:100270007F77709360008FEB17E00E94B20EEEE57F
:10028000F7E20E949A0E709160007F7B709360008D
:1002900000916100083011F00C94600170916000D1
:1002A0007068709360008FEB17E00E94B20EEAE76F
:1002B000F7E20E949A0E709160007F7B709360005D
:1002C00000916100003011F00C9473018FEB17E086
:1002D0000E94B20EE2E8F7E20E949A0E709160006E
:1002E000706470936000009161000C3081E009F04F
:1002F00080E08F930027A0E6B0E08C9186FB0EF49F
:1003000001E041E0041781E009F080E09F9189233A
:10031000882311F40C948E010C940D090091610056
:100320000C3011F00C9496010C949C0184E690E042
:100330000E94610F0C9420010E94A30E84E690E0BD
:100340000E94610F84E08093B1008FE711E00E946A
:10035000B20EECE8F7E20E949A0E8FEB1AE00E94D0
:10036000B20EA8E2B4E0E1EBF0E00E942F130E948D
:10037000920EE0EAF7E20E949A0E8CE00E94100FC3
:100380000E943A0FA1E6B0E00C93009161000430A6
:1003900011F00C94D001A1EBB0E08C918F5F8C93A5
:1003A00000916100083011F00C94DB018091B100E4
:1003B0008A958093B1000091B100013010F00C9447
:1003C000E4018AE08093B1000091B1000A3018F096
:1003D00011F00C94ED010C94F00181E08093B100D8
:1003E000009161000C3011F00C941E020027A0E671
:1003F000B0E08C9187FB0EF401E040E0041711F0AF
:100400000C9409020091B10044E1049FA2EBB0E01A
:100410000C920027A0E6B0E08C9187FB0EF401E07F
:1004200041E0041711F00C941C020091B1004FE060
:10043000049FA2EBB0E00C920C94240284E690E0BE
:100440000E94610F0C94A5010E94A30E84E690E027
:100450000E94610F709160007F7D709360008FE754
:1004600011E00E94B20EE4EAF7E20E949A0E002721
:10047000A0E6B0E08C9185FB0EF401E040E00417AB
:1004800011F00C9450028FEB11E00E94B20EE6EBDB
:10049000F7E20E949A0E8CE00E94100F0C945B020F
:1004A0008FEB11E00E94B20EE6ECF7E20E949A0E8A
:1004B0008CE00E94100F0E943A0FA1E6B0E00C936E
:1004C00000916100043011F00C946B027091600097
:1004D0007F7D7093600000916100083011F00C94F2
:1004E000760270916000706270936000009161000C
:1004F0000C3081E009F080E08F930027A0E6B0E0A7
:100500008C9185FB0EF401E040E0041781E009F0D6
:1005100080E09F918923882311F40C9491020C941C
:10052000B202009161000C3081E009F080E08F930D
:100530000027A0E6B0E08C9185FB0EF401E041E0DD
:10054000041781E009F080E09F918923882311F44A
:100550000C94AC020C945F0784E690E00E94610F5B
:100560000C942F020E94A30E84E690E00E94610F7B
:1005700088EE93E0A5EBB0E08D939C9382E390E04E
:100580009BBD8ABD8FE711E00E94B20EE6EDF7E257
:100590000E949A0E8FEB1AE00E94B20EA8E2B4E01D
:1005A000E5EBF0E00E9420130E94920EE6EEF7E2E7
:1005B0000E949A0E8CE00E94100F0E943A0FA1E652
:1005C000B0E00C9300916100043011F00C94F4023F
:1005D000A5EBB0E00D911C9144E150E0040F151F14
:1005E000A5EBB0E00D931C9300916100083011F071
:1005F0000C940603A5EBB0E00D911C9144E150E092
:10060000041B150BA5EBB0E00D931C93A5EBB0E01C
:100610000D911C91083C50E0150710F00C94160346
:1006200088EB9BE0A5EBB0E08D939C93A5EBB0E04D
:100630000D911C91083B5BE0150718F011F00C942C
:1006400023030C94290388EC90E0A5EBB0E08D9394
:100650009C93009161000C3011F00C944303A5EBC6
:10066000B0E00D911C9144E150E00E94560EA7EBC2
:10067000B0E04D935C9385E390E0A9EBB0E08D93FF
:100680009C930C94490384E690E00E94610F0C94C3
:10069000C20204E813E0A1EBB0E04D9155270E949F
:1006A000700EA3EBB0E00D931C9393980E94A30EE1
:1006B0008FE711E00E94B20EECEEF7E20E949A0E74
:1006C0008CE00E94100F80E087B90E945310A2E6D0
:1006D000B0E08D939C93A2E6B0E00D911C9144E1B3
:1006E00050E00E94700EABEBB0E00D931C93A3EBB7
:1006F000B0E04D915C91ABEBB0E00D911C91041713
:10070000150718F011F00C9487030C948D03AAE4DC
:10071000B0E00E94250E0C949103AAE4B0E00E9480
:100720002B0EAAE4B0E00D911C91043650E01507A1
:1007300018F011F00C949E030C94A20384E690E050
:100740009BBD8ABDA3EBB0E04D915C91ABEBB0E0FB
:100750000D911C910417150781E008F080E08F933C
:10076000AAE4B0E00D911C91053350E0150781E03B
:1007700008F080E09F918923882311F40C94C3032F
:10078000939A0C94E50382E390E00E94610F8FEB53
:1007900011E00E94B20EA8E2B4E0EAE4F0E00E94A8
:1007A00020130E94920EE0EAF7E20E949A0EA8E25D
:1007B000B4E0EBEBF0E00E9420130E94920EE0E028
:1007C000F8E20E949A0E0C94630304EF11E0A1EB8F
:1007D000B0E04D9155270E94700EA5ECB0E00D934E
:1007E0001C93E8E0F7E20E94EE11E5EBF0E0D19017
:1007F000E080FF2400270E94BE100E946311FF27A3
:10080000EDE0ABEEB0E00E947E13ECE0F7E20E9478
:10081000EE11EBEEF0E00E949A100E946311FF27A8
:10082000EDE00E945C10AFEEB0E0DD92EC9285E06E
:1008300085BD979A86E990E00E94610F97980E9483
:10084000A30EE4E0F8E20E949A0E8FEB11E00E9402
:10085000B20EEAE1F8E20E949A0E8CE00E94100FBC
:100860000091B100063018F011F00C9439040C948A
:100870003A04A89A929880E090E09BBD8ABD81E0FE
:1008800080936100A7EBB0E04D915C91A1E6B0E0F0
:100890000D9111270417150718F011F00C9460043E
:1008A000AAE4B0E00E94250E88EC90E00E94610F5F
:1008B000A1E6B0E08C918F5F8C9311F00C94420410
:1008C000A7EBB0E08D919C919BBD8ABD0E94A30EC9
:1008D00080E0809361008FEB11E00E94B20EA8E2ED
:1008E000B4E0EAEEF0E00E942F130E94920EE8E2DC
:1008F000F8E20E949A0EA8E2B4E0E9EEF0E00E946D
:100900002F130E94920EE8E2F8E20E949A0EA8E2EB
:10091000B4E0E8EEF0E00E942F130E94920EEAE2AB
:10092000F8E20E949A0EA8E2B4E0E1EFF0E00E9443
:1009300020130E94920EECE2F8E20E949A0E83E0ED
:100940000E940A0FE2E3F8E20E949A0EA2EDB0E0E4
:100950000E94940EE4E3F8E20E949A0E82E087B9C6
:100960000E945310A3ECB0E08D939C93E0E1F7E27A
:100970000E94EE11E3ECF0E0D190E080FF2400272C
:100980000E94BE100E946311FF27EDE0AFEBB0E0C4
:100990000E947E13E4E1F7E20E94EE11EFEBF0E03B
:1009A0000E949A100E949C11FF27EDE0AFEBB0E08F
:1009B0000E947E13E8E1F7E20E94EE11EFEBF0E017
:1009C0000E949A100E940D11FF27EDE0AFEBB0E0FE
:1009D0000E947E13A8E2B4E0AF93BF93EFEBF0E088
:1009E0000E949A100E94700F112701E0BF91AF91F1
:1009F0000E94D012E8E2F4E0A2EDB0E00E94791388
:100A0000EFEBF0E00E949A10ECE1F7E20E94EE11A9
:100A10000E94F71110F00C941C050E94A30EE8E34D
:100A2000F8E20E949A0E979A88EC90E00E94610F7B
:100A300097988CE00E94100F0091E800063311F0A7
:100A40000C945D07929AA9EBB0E08D919C919BBDAF
:100A50008ABD93980E94A30EEEE4F8E20E949A0EDB
:100A60008FEB11E00E94B20EE0E6F8E20E949A0ECF
:100A70008CE00E94100F0E946B0DAEEFB0E00D9164
:100A80001C91023350E015071CF011F00C944A053C
:100A90000C944B05A99AAEEFB0E00D911C91083271
:100AA00050E015070CF402C00C945705A998E2E039
:100AB000F0E00E94B50E939A85E083BF0091AA00F2
:100AC000003211F00C9466050C9468050C945E05D8
:100AD000882783BF81E08093AA000091AA0000329A
:100AE00018F011F00C949205AAEAB0E0AD90BB2486
:100AF000A2E6B0E0AA0CBB1CAA0DBB1D0D911C9177
:100B0000A4EAB0E04D915C91040F151FA4EAB0E097
:100B10000D931C93AAEAB0E08C918F5F8C9311F037
:100B20000C946D05E0E2F7E20E94EE11E4EAF0E0D9
:100B3000D190E080FF2400270E94BE100E94631124
:100B4000FF27EDE0A6EAB0E00E947E13E6EAF0E0BF
:100B50000E945C10A4EAB0E0DD92EC92E8E1F7E2DA
:100B60000E94EE11E6EAF0E00E949A100E940D1138
:100B7000FF27EDE0A8ECB0E00E947E13A8E2B4E00D
:100B8000AF93BF93E8ECF0E00E949A100E94700FC0
:100B9000112703E0BF91AF910E94D012E8E2F4E088
:100BA000A2EEB0E00E947913A8E2B4E0AF93BF9345
:100BB000E8ECF0E00E949A100E94700F11E002E051
:100BC000BF91AF910E94D012E8E2F4E0ACECB0E04B
:100BD0000E947913A1EFB0E00D911C91AFEEB0E04F
:100BE0004D915C91040F151FA1EFB0E00D931C9384
:100BF000ABEAB0E04D915C91A4EAB0E00D911C919C
:100C00000417150718F011F00C9408060C94100640
:100C1000A4EAB0E08D919C91ABEAB0E08D939C93F7
:100C2000A4EAB0E04D915C91ABEAB0E00D911C916B
:100C30000417150710F40C942B06ABEAB0E00D91E5
:100C40001C91A4EAB0E04D915C91041B150BADEA38
:100C5000B0E00D931C93E8E1F7E20E94EE11EBEA9D
:100C6000F0E0D190E080FF2400270E94BE100E9497
:100C70000D11FF27EDE0A8EDB0E00E947E13A8E281
:100C8000B4E0AF93BF93E8EDF0E00E949A100E94A9
:100C9000700F11E002E0BF91AF910E94D012E8E224
:100CA000F4E0ACEDB0E00E947913A2EBB0E04D911E
:100CB0005527ADEAB0E00D911C910417150710F40B
:100CC0000C94C106A898929A0E94A30E8FE711E097
:100CD0000E94B20EECE6F8E20E949A0EA8E2B4E09E
:100CE000E1EFF0E00E9420130E94920EEAE7F8E2A2
:100CF0000E949A0E8FEB11E00E94B20E80E00E94DB
:100D00000A0FE2E3F8E20E949A0EACECB0E00E9417
:100D1000940EE2E8F8E20E949A0E81E00E940A0F27
:100D2000E2E3F8E20E949A0EACEDB0E00E94940E6D
:100D3000E2E8F8E20E949A0E82E00E940A0FE2E3E3
:100D4000F8E20E949A0EA8E2B4E0EDEAF0E00E9418
:100D500020130E94920EE4E8F8E20E949A0EE8E85E
:100D6000F8E20E94840E0E948B0E8CE00E94100F0D
:100D7000F894979AE1E0F0E00E94B50E9798F89405
:100D8000FFCFA5ECB0E04D915C91A4EAB0E00D91ED
:100D90001C910417150710F00C94D306A7ECB0E0D3
:100DA0008C918F5F8C930091C700033011F00C94ED
:100DB000FB06929AA8980E94A30EE6E9F8E20E9428
:100DC0009A0E0E94A10EE8EAF8E20E949A0EACEC9C
:100DD000B0E00E94940EE4EBF8E20E949A0E8CE0E0
:100DE0000E94100FF894979AE1E0F0E00E94B50E8F
:100DF0009798F894FFCF0E94A30E80E00E940A0FFC
:100E0000E2E3F8E20E949A0EACECB0E00E94940E8D
:100E1000E2E8F8E20E949A0E81E00E940A0FE2E303
:100E2000F8E20E949A0EACEDB0E00E94940EE2E867
:100E3000F8E20E949A0E82E00E940A0FE2E3F8E2D2
:100E40000E949A0EA8E2B4E0EDEAF0E00E942013BE
:100E50000E94920EE4E8F8E20E949A0EA2EEB0E040
:100E60000E947E0EE0EAF7E20E94840EA8E2B4E05F
:100E7000E4EAF0E00E9420130E947C0E80E0809360
:100E8000AA0080E090E0A4EAB0E08D939C93A6EAEB
:100E9000B0E0E4E2F7E20E941E0E979A81E090E053
:100EA0000E94610F97988CE00E94100FA7EBB0E0B2
:100EB0008D919C919BBD8ABD92980C946B0480E0AF
:100EC0008093AA000E94A30E84E690E00E94610F26
:100ED00084E690E0A5EBB0E08D939C9383E090E0F6
:100EE0009BBD8ABD8FE711E00E94B20EE6EDF7E2EE
:100EF0000E949A0E8FEB1AE00E94B20EA8E2B4E0B4
:100F0000E5EBF0E00E9420130E94920EE6EEF7E27D
:100F10000E949A0E8CE00E94100F0E943A0FA1E6E8
:100F2000B0E00C9300916100043011F00C94A40720
:100F3000A5EBB0E00D911C9144E150E0040F151FAA
:100F4000A5EBB0E00D931C9300916100083011F007
:100F50000C94B607A5EBB0E00D911C9144E150E074
:100F6000041B150BA5EBB0E00D931C93A5EBB0E0B3
:100F70000D911C91083250E0150710F00C94C60733
:100F800080E491E0A5EBB0E08D939C93A5EBB0E0FD
:100F90000D911C91003451E0150718F011F00C94DC
:100FA000D3070C94D90788E290E0A5EBB0E08D93CD
:100FB0009C93009161000C3011F00C94FB07A5EBA1
:100FC000B0E00D911C9144E150E00E94560EA7EB59
:100FD000B0E04D935C93A7EBB0E00D911C9142E023
:100FE00050E0041B150BBB27A0E18D919C919BBD8C
:100FF0008ABD0C94010884E690E00E94610F0C9475
:10100000720780E08093610092980091B1000630F1
:1010100018F011F00C940E080C940F08A89A85E0B3
:1010200085BD0E94A30E8FE711E00E94B20EE8EB8F
:10103000F8E20E949A0E8FEB11E00E94B20EA8E235
:10104000B4E0EAEEF0E00E942F130E94920EE8E274
:10105000F8E20E949A0EA8E2B4E0E9EEF0E00E9405
:101060002F130E94920EE8E2F8E20E949A0EA8E284
:10107000B4E0E8EEF0E00E942F130E94920EEEEC36
:10108000F8E20E949A0E80E00E940A0FE2EDF8E278
:101090000E949A0EACECB0E00E94940EE6EDF8E2ED
:1010A0000E949A0E8CE00E94100F0091E800093314
:1010B00011F00C94F30885E083BF0E94A30E8FE724
:1010C00017E00E94B20EECEDF8E20E949A0E8CE05E
:1010D0000E94100F80E090E0A4EAB0E08D939C9312
:1010E000A6EAB0E0E4E2F7E20E941E0E0091AA0038
:1010F000003211F00C947E080C9480080C94760851
:10110000882783BF81E08093AA000091AA00003263
:1011100018F011F00C94AA08AAEAB0E0AD90BB2434
:10112000A2E6B0E0AA0CBB1CAA0DBB1D0D911C9140
:10113000A4EAB0E04D915C91040F151FA4EAB0E061
:101140000D931C93AAEAB0E08C918F5F8C9311F001
:101150000C948508E0E2F7E20E94EE11E4EAF0E088
:10116000D190E080FF2400270E94BE100E946311EE
:10117000FF27EDE0A6EAB0E00E947E13E6EAF0E089
:101180000E945C10A4EAB0E0DD92EC92E8E1F7E2A4
:101190000E94EE11E6EAF0E00E949A100E940D1102
:1011A000FF27EDE0A8ECB0E00E947E13A8E2B4E0D7
:1011B000AF93BF93E8ECF0E00E949A100E94700F8A
:1011C000112702E0BF91AF910E94D012E8E2F4E053
:1011D000ACECB0E00E947913ACECB0E00E947E0E63
:1011E00080E08093AA000091EA000F3011F00C9487
:1011F0000B09F8940E94A30E8FE711E00E94B20E33
:10120000E8EEF8E20E949A0E8CE00E94100FA89877
:10121000929AF894FFCF0C9413080E94A30E84E6D0
:1012200090E00E94610F82E08093B1008FE711E0AF
:101230000E94B20EE8EFF8E20E949A0E8FEB1AE0DD
:101240000E94B20EA8E2B4E0E1EBF0E00E942F139E
:101250000E94920EE0E1F9E20E949A0E8CE00E9458
:10126000100F0E943A0FA1E6B0E00C9300916100CC
:10127000043011F00C944109A1EBB0E08C918F5F28
:101280008C9300916100083011F00C944C0980910E
:10129000B1008A958093B1000091B100013010F047
:1012A0000C94550981E08093B1000091B1000330A6
:1012B00018F011F00C945E090C94610983E080939E
:1012C000B100009161000C3011F00C9469090C948C
:1012D0006F0984E690E00E94610F0C9416090E9449
:1012E000A30E84E690E00E94610F88EE93E0A5EBE8
:1012F000B0E08D939C9382E390E09BBD8ABD8FE725
:1013000011E00E94B20EE6EDF7E20E949A0E8FEB1A
:101310001AE00E94B20EA8E2B4E0E5EBF0E00E9411
:1013200020130E94920EE6EEF7E20E949A0E8CE0E5
:101330000E94100F0E943A0FA1E6B0E00C930091BA
:101340006100043011F00C94B109A5EBB0E00D91EF
:101350001C9144E150E0040F151FA5EBB0E00D9384
:101360001C9300916100083011F00C94C309A5EBA7
:10137000B0E00D911C9144E150E0041B150BA5EB6E
:10138000B0E00D931C93A5EBB0E00D911C91083CCF
:1013900050E0150710F00C94D30988EB9BE0A5EB07
:1013A000B0E08D939C93A5EBB0E00D911C91083BB0
:1013B0005BE0150718F011F00C94E0090C94E609B5
:1013C00088EC90E0A5EBB0E08D939C9300916100D8
:1013D0000C3011F00C94FA09A5EBB0E00D911C91C2
:1013E00044E150E00E94560EA7EBB0E04D935C93B1
:1013F0000C94000A84E690E00E94610F0C947F092F
:101400000091B100013011F00C94070ADB9A0091B1
:10141000B100023011F00C940E0ADC9A0091B10078
:10142000033011F00C94170ADD9A909AA89AA7EB52
:10143000B0E08D919C919BBD8ABD0E94A30EE4E01B
:10144000F8E20E949A0E8FEB11E00E94B20EEAE1E0
:10145000F8E20E949A0E8CE00E94100F85E085BD94
:10146000929880E090E09BBD8ABD81E0809361000E
:10147000A7EBB0E04D915C91A1E6B0E00D91112792
:101480000417150718F011F00C94560AAAE4B0E0FE
:101490000E94250E88EC90E00E94610FA1E6B0E06A
:1014A0008C918F5F8C9311F00C94380AA7EBB0E00D
:1014B0008D919C919BBD8ABD979A86E990E00E9490
:1014C000610F979880E08093610080E090E0A4EA4B
:1014D000B0E08D939C9380E08093AA0080E090E040
:1014E000ABEAB0E08D939C9380E08093E80080E0CD
:1014F0008093E90080E08093EA000E94A30E82E0DE
:1015000087B90E945310A3ECB0E08D939C93E0E167
:10151000F7E20E94EE11E3ECF0E0D190E080FF24CE
:1015200000270E94BE100E946311FF27EDE0AFEB81
:10153000B0E00E947E13E4E1F7E20E94EE11EFEBCF
:10154000F0E00E949A100E949C11FF27EDE0AFEBA3
:10155000B0E00E947E13E8E1F7E20E94EE11EFEBAB
:10156000F0E00E949A100E940D11FF27EDE0AFEB12
:10157000B0E00E947E13A8E2B4E0AF93BF93EFEB1C
:10158000F0E00E949A100E94700F112701E0BF91B5
:10159000AF910E94D012E8E2F4E0A2EDB0E00E9428
:1015A0007913EFEBF0E00E949A10ECE1F7E20E9471
:1015B000EE110E94F71110F00C94ED0A0E94A30E98
:1015C000E8E3F8E20E949A0E979A8AEF90E00E9470
:1015D000610F97988CE00E94100F0091E80006338D
:1015E00011F00C946B0C0E94A30EEEE4F8E20E9442
:1015F0009A0E8FEB11E00E94B20EE0E6F8E20E9434
:101600009A0E8CE00E94100F0E946B0DAEEFB0E0BE
:101610000D911C91023350E015071CF011F00C9451
:10162000130B0C94140BA99AAEEFB0E00D911C9122
:10163000083250E015070CF402C00C94200BA99856
:1016400081E08093B00085E083BF0091AA00003262
:1016500011F00C942D0B0C942F0B0C94250B882758
:1016600083BF81E08093AA000091AA00003218F0A5
:1016700011F00C94590BAAEAB0E0AD90BB24A2E69D
:10168000B0E0AA0CBB1CAA0DBB1D0D911C91A4EAD5
:10169000B0E04D915C91040F151FA4EAB0E00D93EA
:1016A0001C93AAEAB0E08C918F5F8C9311F00C949C
:1016B000340BE8E2F7E20E94EE11E4EAF0E0D190A8
:1016C000E080FF2400270E94BE100E946311FF27C4
:1016D000EDE0A6EAB0E00E947E13E6EAF0E00E94A8
:1016E0005C10ADEBB0E0DD92EC9280E08093AA005C
:1016F00080E090E0A4EAB0E08D939C93A6EAB0E08D
:10170000E4E2F7E20E941E0E929A80E08093B0001D
:1017100085E083BF0091AA00003211F00C94920B77
:101720000C94940B0C948A0B882783BF81E08093E0
:10173000AA000091AA00003218F011F00C94BE0B20
:10174000AAEAB0E0AD90BB24A2E6B0E0AA0CBB1CB4
:10175000AA0DBB1D0D911C91A4EAB0E04D915C91C6
:10176000040F151FA4EAB0E00D931C93AAEAB0E0A1
:101770008C918F5F8C9311F00C94990BE0E2F7E25F
:101780000E94EE11E4EAF0E0D190E080FF2400270F
:101790000E94BE100E946311FF27EDE0A6EAB0E0B0
:1017A0000E947E13E6EAF0E00E945C10A4EAB0E03A
:1017B000DD92EC92E8E1F7E20E94EE11E6EAF0E059
:1017C0000E949A100E940D11FF27EDE0A8ECB0E0F6
:1017D0000E947E13A8E2B4E0AF93BF93E8ECF0E080
:1017E0000E949A100E94700F11E002E0BF91AF9129
:1017F0000E94D012E8E2F4E0ACECB0E00E94791371
:1018000080E08093AA0080E090E0A4EAB0E08D93AD
:101810009C93A6EAB0E0E4E2F7E20E941E0E0E946A
:10182000A30E8FE711E00E94B20E80E00E940A0F23
:10183000E2E3F8E20E949A0EACECB0E00E94940E53
:10184000E4E1F9E20E949A0EA8E2B4E0EDEBF0E0E8
:101850000E9420130E94920EEEE1F9E20E949A0E7D
:10186000979A81E090E00E94610F97989298ADEB73
:10187000B0E00D911C91023350E0150710F00C946C
:101880006B0C9098A898929A0E94A30EE4E2F9E259
:101890000E949A0E8FEB11E00E94B20EA8E2B4E013
:1018A000EAEEF0E00E942F130E94920EEEE3F9E2BE
:1018B0000E949A0EA8E2B4E0E9EEF0E00E942F1335
:1018C0000E94920EE2E4F9E20E949A0E8CE00E94DD
:1018D000100FF894FFCF8FEB11E00E94B20EA8E238
:1018E000B4E0EAEEF0E00E942F130E94920EE8E2CC
:1018F000F8E20E949A0EA8E2B4E0E9EEF0E00E945D
:101900002F130E94920EE8E2F8E20E949A0EA8E2DB
:10191000B4E0E8EEF0E00E942F130E94920EEEEC8D
:10192000F8E20E949A0E83E00E940A0FE2E3F8E2D6
:101930000E949A0EA2EDB0E00E94940EE4E3F8E259
:101940000E949A0E8CE00E94100F0C947F0A0F9256
:101950001F922F923F924F925F927F928F929F920F
:10196000AF92BF920F931F932F933F934F935F9329
:101970006F937F938F939F93AF93BF93CF93DF9397
:10198000EF93FF938FB78F93A1E6B0E08C918F5FB9
:101990008C9300916100033011F00C94F10CAAEAD1
:1019A000B0E08C918F5F8C93A0EBB0E08C9187B905
:1019B0000E945310A2E6B0E08D939C93A2E6B0E0A3
:1019C0008D919C91AAEAB0E0AD90BB24A2E6B0E074
:1019D000AA0CBB1CAA0DBB1D8D939C9380E0809329
:1019E00061008F918FBFFF91EF91DF91CF91BF91F8
:1019F000AF919F918F917F916F915F914F913F91A7
:101A00002F911F910F91BF90AF909F908F907F90DB
:101A10005F904F903F902F901F900F9018950F92CE
:101A20001F922F923F924F925F927F928F929F923E
:101A3000AF92BF920F931F932F933F934F935F9358
:101A40006F937F938F939F93AF93BF93CF93DF93C6
:101A5000EF93FF938FB78F93A8EEB0E08C918F5FD9
:101A60008C930091E8000C3311F00C943F0D80E052
:101A70008093E800A9EEB0E08C918F5F8C93009189
:101A8000E9000C3311F00C944D0D80E08093E900D7
:101A9000AAEEB0E08C918F5F8C938F918FBFFF91F6
:101AA000EF91DF91CF91BF91AF919F918F917F91F6
:101AB0006F915F914F913F912F911F910F91BF9027
:101AC000AF909F908F907F905F904F903F902F901E
:101AD0001F900F90189586E0E0E30E942F126CECA7
:101AE00086E0E0E3BB27A6E121E02A930E94621290
:101AF00064E486E0E0E3BB27A6E121E02A930E94AC
:101B00006212E1E0F0E00E94B50E86E0E0E30E94A0
:101B10002F126CEC86E0E0E3BB27A6E121E02A93DC
:101B20000E9462126EEB86E0E0E3BB27A6E121E0B3
:101B30002A930E94621286E0A3EFB0E0E0E329E07E
:101B40002A930E949E1286E0E0E30E942F120091E9
:101B5000F30041E00423ADEFB0E00C930091FD00F1
:101B6000013011F00C94B90D8091F3008A958093A7
:101B7000F300A4EFB0E09C91A3EFB0E08C91AEEF46
:101B8000B0E08D939C93AEEFB0E00D911C9142E3D9
:101B900050E00E94310EAEEFB0E00D931C93AEEF1B
:101BA000B0E00D911C9149E150E0041B150BAEEF24
:101BB000B0E00D931C93AAEFB0E00D911127A9EFAF
:101BC000B0E04D915527041B150BA0E0B1E00D933B
:101BD0001C93A0E0B1E00D911C9144E650E00E94FE
:101BE000310EA0E0B1E00D931C93A0E0B1E00D91A7
:101BF0001C91AAEFB0E04D9155270E94360EA0E04F
:101C0000B1E04D935C93AEEFB0E00D911C91A0E07C
:101C1000B1E04D915C91040F151FAEEFB0E00D9354
:101C20001C93AEEFB0E00D911C9144E650E00E9491
:101C3000360EAEEFB0E04D935C93089584E0C89506
:101C400031960D928A95D9F70895ED91FC913196D0
:101C5000FC93EE930895ED91FC913197FC93EE93F4
:101C6000089508D03DD000FC10D0089503D01ED0B8
:101C700001F8F9CF0024E89457FF02C009D0689416
:101C800000F80BD010F80124089502D009D008956F
:101C9000509540954F5F5F4F0895E89417FF089562
:101CA000009510950F5F1F4F68940895352F242FCE
:101CB000E894452B11F468940895512F402F002784
:101CC000112780E1440F551F001F111F021B130B2A
:101CD000416018F4020F131F4E7F8A9599F70895FB
:101CE0000F92049F202C312C419F300C509F030CED
:101CF000022D102D0F900895A8E2B4E08D91882355
:101D000011F00CD0FBCF08950E94EA11802D11F044
:101D100005D0FACF08958DE001D08AE05D9BFECF1B
:101D20008CB90895A8E2B4E08D91882311F072D0A7
:101D3000FBCF08950E94EA11802D11F06BD0FACFED
:101D4000089580EC6DC081E06BD015D080E868C04C
:101D50008FE7213039F08FEB223021F08FE82330EC
:101D600009F08FEC810F0C94100F88EE93E0A9D04E
:101D70003197D9F7089583E09927A3C08AEF90E0BF
:101D80000E94610FA59AA49AA39AA29AD69AD79A6A
:101D9000DF98EF93FF93E4ECF0E00E94310FFF91A6
:101DA000EF91DE98AD98AC98AB9AAA9ADE9AEF9331
:101DB000FF93E4ECF0E00E94310FFF91EF91DE9889
:101DC0007DD0DE9AEF93FF93E4ECF0E00E94310FB8
:101DD000FF91EF91DE9872D0DE9AEF93FF93E4ECDF
:101DE000F0E00E94310FFF91EF91DE9867D0AA9842
:101DF000DE9AEF93FF93E4ECF0E00E94310FFF9145
:101E0000EF91DE985BD088E20BD08EE009D086E0BF
:101E100007D00895DF9A829505D004D04FD0089559
:101E2000DF98F9CF859510F4AA9A01C0AA988595F4
:101E300010F4AB9A01C0AB98859510F4AC9A01C030
:101E4000AC98859510F4AD9A01C0AD98DE9AEF93E9
:101E5000FF93E4ECF0E00E94310FFF91EF91DE98E8
:101E600008953197F1F70895689462F80895E89419
:101E700062F8089500E18FEF88BB8FE087BB80EFA9
:101E800088BB84E18A95F1F7B49B00E0B59B04E040
:101E9000B69B08E0B79B0CE080EF87BB8FE088BB68
:101EA00084E18A95F1F78827B09B80E0B19B81E0BF
:101EB000B29B82E0B39B83E0080F089581E090E03D
:101EC00000C0EF93FF93EE27E82BE92B31F0E0ED14
:101ED000F7E03197F1F70197D1F7FF91EF9108956E
:101EE0008DE207FD8D938F2D881F802F881F8F57C0
:101EF000082F6894F7F8802F87FF15C08095839589
:101F0000082F80E38D938EE28D93802F815228F0ED
:101F100080E38D9399279C93089544270A95802FF9
:101F200009F196D01FC0805230F09EE49D9381E469
:101F30008D939D93EFCF4427DF92EF92FF920F9303
:101F40008FE1801B11F0082F83D089D09EE29D93F2
:101F50000F91FF90EF90DF9044270395003209F432
:101F6000D7CF2BD03F93E0EFFFE138E12F2D1E2D8F
:101F70000D2DFF24EE24DD244427000F111F221F06
:101F8000A8F42F923F920E94EA11102C0E94EA11AD
:101F9000202C0E94EA11302C0E94EA113197410D49
:101FA000D21CE31CF01C3F902F9001C03396319659
:101FB0003A9519F73F9107D0AFCFDD0CEE1CFF1C0F
:101FC0000A95D9F70895002719E058D08F93802BF0
:101FD00011F0039501C08F911A95B9F7802F8823CE
:101FE00009F496CF8F91805D8D930A95D9F792CFA2
:101FF0000065CD1D80B2E60E40597307A0ACB90351
:1020000050D6DC01286BEE0094357700CA9A3B006D
:1020100065CD1D00B2E60E0059730700ACB9030090
:10202000D6DC01006BEE0000357700009A3B000023
:10203000CD1D0000E60E000073070000B90300008C
:10204000DC010000EE000000770000003B00000013
:10205000F694E794D79447950A95D1F70895002709
:102060000DD08F9303958F2D8E298D29842BC1F749
:102070008F91805D8D930A95D9F74CCF1F930F9365
:10208000002710E2440FDD1CEE1CFF1C001F802FF8
:102090009AE0890B10F0082F43951A9599F7802F35
:1020A0000F911F910895369A3699FECF369A369938
:1020B000FECF84B195B108953DD0992711278F2D7A
:1020C000880F80E8F82A802F881F08F41FEF41F05E
:1020D0008F57082F07FD04C0003240F08FEF01C07A
:1020E0008827982FD82EE82EF82E09C08FE1801B64
:1020F000082FF694E794D79497950A95D1F7112372
:1021000051F09095D094E094F09481E0980F882756
:10211000D81EE81EF81E0F2DFE2CED2CD92E08958A
:10212000D094E094F09491E0D90E9927E91EF91E1D
:1021300010950895D190E190F19001910895219129
:102140003191419151910895102F90E8FF0C001F9B
:102150000927990FF7941078652F90E8440F551FC1
:102160005927990F4795607800380895FF0C90E83B
:102170009027110F9795F794092F0895112707FBC2
:1021800056F4D094E094F094009591E0D90EE11EBD
:10219000F11E011F1FEF9FE1DD0CEE1CFF1C001F55
:1021A00007FD07C09A95C1F7EE24FF240027992761
:1021B0000DC09258D7FA56F4E39440F40024F01C72
:1021C000001D20F493950795F794E794DE2CEF2CEF
:1021D000F02E110F9795092F10F4689401C0E89420
:1021E000F7F80895502F2D2D3E2D4F2D612F089576
:1021F0002DEC3CEC4CEC5DE366270FC09BDFF2DF7F
:10220000DD24EE2490E8F92E0FE307C098DF05C027
:102210002227332740E251E46627552351F100235A
:1022200081F192DF71F11627005850580894050B80
:1022300018F407FD03C025C007FD23C04695379558
:102240002795F694E794D79422D0FF202AF0DD0C4E
:10225000EE1CFF1C015073F09D2D969548F0DD207B
:102260003AF4EE202AF491E0D90E9927E91EF91EDE
:102270007DCF07C09FE7092FF92A9FEFD92EE92EBE
:102280000895DD24EE24FF240027112708959F924E
:102290009924AA24BB2488E1D216E306F40628F088
:1022A000D21AE30AF40A089401C08894991CAA1C63
:1022B000BB1CDD0CEE1CFF1C8A9571F7D92CEA2C97
:1022C000FB2C9F90089540DFE1F25038D1F21627A1
:1022D000005850580894051F12F418F4CBCF08F09A
:1022E000D0CF0AD0FF202AF0BB0CDD1CEE1CFF1C57
:1022F0003DCF0F5FFBF13ACF9F929924AA24BB24D4
:10230000992788E1990CAA1CBB1CDD1CEE1CFF1C44
:1023100030F4920EA31EB41ED91EE91EF91E8A9532
:1023200089F79F9008950AF045D020CF5FE32227D8
:102330003327442701C003DF07DF5038B1F30038EB
:1023400099F3902F951B8BF312F434D0FACF983178
:1023500018F0222733274427983028F0232F342FD2
:1023600044279850F9CF992329F04695379527951A
:102370009A95D9F7912F962742F014D0B0F6F7949A
:10238000E794D7940F5F8BF675CF10D051F008F417
:10239000C7DEFF2052F2DD0CEE1CFF1C0150CBF714
:1023A00069CF6FCFD20EE31EF41E0895D21AE30A4E
:1023B000F40A0895DF92EF92FF920F931F93D22EAB
:1023C000E32EF42E052F162F6F915F914F913F91C1
:1023D0002F910895C895319600200895FBDF202D98
:1023E000F9DF302DF7DF402DF5DF502D089507FB85
:1023F00000680EF40F7757FB50680EF45F7707FD07
:1024000002C057FF05C0D216E306F406050708957B
:102410002D153E054F055007089591E0882321F0C2
:102420008894991F8A95E9F7892F909508950181DD
:10243000082B018312811923128300000000000081
:10244000000000000000000000000000000000008C
:1024500000000000000000000000000008950E943D
:10246000340FFF270E940D12E2DFEF93FF93ECEB96
:10247000F3E00E94310FFF91EF91182B1283092393
:102480000183EF93FF93E0EBF0E00E94310FFF91A7
:10249000EF911081182369F4EF93FF93ECEBF3E0D5
:1024A0000E94310FFF91EF911081182311F00E94CB
:1024B000370FEF93FF93ECEBF3E00E94310FFF91A6
:1024C000EF9108950E940D12FF2729915D9148E038
:1024D000AEDF00000000000000000000000000006F
:1024E00000000000000000000000000000000000EC
:1024F00000000000579510F4182B1283EF93FF9300
:10250000E4E7F0E00E94310FFF91EF91182B128366
:1025100000000000000000000000000000000000BB
:1025200000000000000000000000000000000000AB
:1025300000004A9569F62A9549F608950E940D1201
:10254000FF27299148E0552772DF09230183EF9384
:10255000FF93E8E0F0E00E94310FFF91EF91889443
:102560001081182309F008945795EF93FF93E6E53F
:10257000F0E00E94310FFF91EF914A9529F75D93AA
:102580002A9501F7089599278D9193958823E1F76E
:10259000939511968C9311978E919A95D1F70895F2
:1025A000EA2FFB2F00248D9103948E32E1F7112442
:1025B0008D9113948823E1F71A94101640F4119723
:1025C000202F2119239580E38D932A95E9F7113067
:1025D00011F59927AE2FFF2FA00DB91FA00FB91F1E
:1025E0008C919C93853308F41CC031E08E918E321F
:1025F000E9F3830F8A3319F480E331E001C0332714
:102600008C93AE1799F7332329F0AE2FBF2FBBDF82
:1026100081E3808308958827E00DF81FE00FF81FFD
:1026200080830895000F111F221F331F0895009506
:102630001095209530950F5F1F4F2F4F3F4F0895F6
:10264000019110810EC001911191219130810BC037
:102650000191108117FF05C03FEF2FEF04C00081EB
:1026600011272227332737FF03C0E1DF8DE28D9347
:10267000CF93DF93CF92DF92EF92AA24BB24CC2496
:10268000DD24EE2440E2CAE0DD2755E093E38881B3
:10269000890F87FD9F7083FD907F891B89935A95D1
:1026A000A9F7C0DFAA1CBB1CCC1CDD1CEE1C4A9584
:1026B00051F7E894EFE0FF2782910ED0EB30E0F77E
:1026C0001EF068948A2D0CD088278D93EF90DF90B0
:1026D000CF90DF91CF910895982F829501D0892FC7
:1026E0008F70805D26F0803309F4089568948D938F
:1026F000089581918D938823E1F7089594E0819165
:102700008D939A95E1F708956666663F96438B3CF4
:102710000000A04100002F4400007A44CDCC344199
:102720000000203F000000000000003E2A2A2A206E
:102730004C4154414E4945204E41204C555A494543
:10274000202A2A2A000020202020207777772E6157
:102750006C657872632E636F6D2020200000204E20
:10276000694364202000506F64616A20747970208E
:102770006F676E6977613A200000204E694D6820CE
:102780002000204C69496F6E20200000506F64616A
:102790006A20696C6F7363206F676E69773A2000F7
:1027A00020200000437A6173206C61646F77616E52
:1027B00069613A20000042657A206C696D69747520
:1027C0002020202000004C61646F77616E696520D5
:1027D0003135682000004F6B7265736C2070726138
:1027E000643A202000006D4120200000547277617F
:1027F00020726F7A6C61646F777977616E696500BA
:1028000020202000557374616C616E6965207061D1
:1028100072616D6574726F7720006C61646F7761AF
:102820006E696120202000003A002A006D41682A6C
:1028300000003D0056200000534C41425920414BBE
:10284000554D554C41544F522021212100005452E6
:102850005741204F44435A59545957414E49450016
:10286000504152414D4554524F5700004B6F6E69D5
:1028700065632020506F6A3A0000206D4168202077
:10288000200056006D5620002A2A2A6B6F6E69655B
:10289000632A2A2A000055737A6B6F647A6F6E7907
:1028A0002070616B696574004E617069656369656C
:1028B0003D2000002056000054525741204C414416
:1028C0004F57414E49452031356820200000202ACD
:1028D00020003D2000002056202020005452574167
:1028E00020504F4D494152004B6F6E696563206C1B
:1028F00061642E2031356800506F64616A20726F08
:10290000647A616A2070616B696574753A200000B1
:102910005320200056202A20507261643D00206D13
:10292000412000004C61646F77616E6965207A61B7
:102930006B6F6E637A6F6E6520706F3A000068206F
:042940003A006D00EC
:00000001FF
